:020000040000FA
:1000000000700020250400003704000039040000BF
:100010003B0400003D0400003F040000000000001D
:10002000000000000000000000000000410400008B
:1000300043040000000000004504000025150000F6
:10004000490400004904000049040000490400007C
:10005000490400004904000049040000490400006C
:10006000490400004904000049040000490400005C
:10007000490400004904000049040000490400004C
:10008000490400004904000049040000490400003C
:10009000490400004904000049040000490400002C
:1000A000490400004904000049040000490400001C
:1000B000850F0000490400004904000049040000C5
:1000C00049040000490400004904000049040000FC
:1000D00049040000490400004904000049040000EC
:1000E00049040000490400004904000049040000DC
:1000F00049040000490400004904000049040000CC
:10010000990D000049040000490400004904000062
:1001100049040000490400004904000049040000AB
:10012000490400004904000049040000490400009B
:10013000490400004904000035120000711200005B
:10014000490400004904000049040000490400007B
:10015000490400004904000049040000490400006B
:10016000490400004904000049040000490400005B
:10017000490400004904000049040000490400004B
:1003F000490400004904000049040000FFFFFFFF1A
:020000040000FA
:10040000FFFFFFFFFFFFFFFFFFFFFFFFFE7FFFFF7D
:020000040000FA
:10041000DFF80CD000F022F800480047991D0000DA
:1004200000700020094872B6094880470948804793
:1004300062B609480047FEE7FEE7FEE7FEE7FEE793
:10044000FEE7FEE7FEE7FEE7FEE70000000400002F
:10045000FD170000291B000011040000064C074D89
:1004600006E0E06840F0010394E807009847103484
:10047000AC42F6D3FFF7D0FF781E0000981E0000B4
:1004800070B58C1810F8015B15F0070301D110F856
:10049000013B2A1106D110F8012B03E010F8016B83
:1004A00001F8016B5B1EF9D12B0705D40023521E06
:1004B0000DD401F8013BFAE710F8013BCB1A921C6E
:1004C00003E013F8015B01F8015B521EF9D5A1426C
:1004D000D8D3002070BD00001248006820F0804092
:1004E0001049EC39C1F8EC000846D0F8EC0040F0B7
:1004F0008070C1F8EC000846D0F8EC0040F0804075
:10050000084908601F2008490860042008640C207E
:10051000486400200449903108600349C1F8940000
:1005200070470000EC50064000B00340F848408D92
:10053000F8490880F64840894880F548B0F8A80096
:100540008880F348B0F88800C880F148B0F86800A7
:100550000881EF48B0F848004881ED48008D888157
:10056000EB480089C881EA48B0F8A6000882E8484C
:10057000B0F886004882E648B0F866008882E44811
:10058000B0F84600C882E248C08C0883E048C088C2
:100590004883DF48B0F8A4008883DD48B0F88400C1
:1005A000C883DB48B0F864000884D948B0F8441028
:1005B000D8484184D648818CD6488184D4488188E3
:1005C000D448C184D248B0F8A210D2480185D0489E
:1005D000B0F88210CF484185CD48B0F86210CD48C0
:1005E0008185CB48B0F84210CA48C185C848418CC3
:1005F000C8480186C6484188C6484186C448B0F804
:10060000A010C4488186C248B0F88010C148C18695
:10061000BF48B0F86010BF480187BD48B0F840102F
:10062000BC484187BA48018CBA488187B8480188DC
:10063000B848C187B648B0F8AE00B649A1F8400046
:10064000B348B0F88E10B348A0F84210B048B0F8E4
:100650006E10B048A0F84410AD48B0F84E10AD4848
:10066000A0F84610AA48C18DAA48A0F84810A8488A
:10067000C189A848A0F84A10A548B0F8AC10A54810
:10068000A0F84C10A248B0F88C10A248A0F84E1068
:100690009F48B0F86C109F48A0F850109C48B0F8E4
:1006A0004C109C48A0F852109948818D9948A0F8A8
:1006B0005410974881899748A0F856109448B0F88C
:1006C000AA109448A0F858109148B0F88A109148A0
:1006D000A0F85A108E48B0F86A108E48A0F85C1046
:1006E0008B48B0F84A108B48A0F85E108848408FBD
:1006F0008849A1F860008648418B8648A0F86210BE
:100700008348B0F8B8108348A0F864108048B0F867
:1007100098108048A0F866107D48B0F878107D48A1
:10072000A0F868107A48B0F858107A48A0F86A1013
:100730007748018F7748A0F86C107548018B754891
:10074000A0F86E107248B0F8B6107248A0F8701099
:100750006F48B0F896106F48A0F872106C48B0F867
:1007600076106C48A0F874106948B0F856106948C3
:10077000A0F876106648C18E6648A0F878106448E4
:10078000C18A6448A0F87A106148B0F8B410614892
:10079000A0F87C105E48B0F894105E48A0F87E1077
:1007A0005B48B0F8BE005B49A1F880005848B0F83B
:1007B0009E105848A0F882105548B0F87E10554851
:1007C000A0F884105248B0F85E105248A0F8861085
:1007D0004F48C18F4F48A0F888104D48C18B4D48F5
:1007E000A0F88A104A48B0F8BC104A48A0F88C100B
:1007F0004748B0F89C104748A0F88E104448B0F81D
:100800007C104448A0F890104148B0F85C10414872
:10081000A0F892103E48818F3E48A0F894103C48C2
:10082000818B3C48A0F896103948B0F8BA10394886
:10083000A0F898103648B0F89A103648A0F89A10E8
:100840003348B0F87A103348A0F89C103048B0F81C
:100850005A103048A0F89E102D48B0F874002D4969
:10086000A1F8A0002A48B0F854102A48A0F8A21015
:100870002748818E2748A0F8A4102548818A25485A
:10088000A0F8A6102248B0F8B2102248A0F8A8108C
:100890001F48B0F892101F48A0F8AA101C48B0F8E2
:1008A00072101C48A0F8AC101948B0F85210194842
:1008B000A0F8AE101648418E1648A0F8B0101448A3
:1008C000418A1448A0F8B2101148B0F8B01011488D
:1008D000A0F8B4100E48B0F890100E48A0F8B6106A
:1008E0000B48B0F870100B48A0F8B8100848B0F8E2
:1008F00050100848A0F8BA100548018E0548A0F825
:10090000BC100348018A0348A0F8BE1070470000DD
:10091000EC82FF1F6C85FF1F002011E000210BE01F
:1009200000224FF47A7392FBF3F2074B03EB401370
:1009300023F811204A1CD1B21029F1DB421CD0B29D
:100940000628EBDB704700006C85FF1F002015E0D8
:1009500000210FE00B4A128840F604535A434FF42B
:100960007A7392FBF3F2084B03EB401323F8112048
:100970004A1CD1B21029EDDB421CD0B20628E7DBBD
:10098000704700006C80FF1F6C85FF1F10B54F483B
:100990000078042802D04E48007860B900204D4904
:1009A00008704D4800780978884232D0494800786C
:1009B000494908702DE04548007898B944480078C6
:1009C00001280FD14548007860B9012041490870DD
:1009D00041480078097888421BD03E4800783E495B
:1009E000087016E03948007898B93948007801282D
:1009F0000FD13A48007801280BD102203549087000
:100A0000354800780978884203D032480078324966
:100A1000087033480078002857D1324800880328EE
:100A20004BDA0F2361220121084600F0B1FF0F23AA
:100A300061220221012000F0ABFF0F23612203217C
:100A4000012000F0A5FF0F2361220121022000F008
:100A50009FFF0F2361220221084600F099FF0F2318
:100A600061220321022000F093FF00236122012173
:100A7000084600F08DFF002361220221012000F0D2
:100A800087FF002361220321012000F081FF002362
:100A900061220121022000F07BFF0023612202215C
:100AA000084600F075FF002361220321022000F0B8
:100AB0006FFF01200A49087002E0032009490880FD
:100AC00008480088401C0749088010BD4680FF1F69
:100AD0003A80FF1F0180FF1F0080FF1F4080FF1F23
:100AE0006F80FF1F7480FF1F28210248416401218D
:100AF00081647047006002400E48006820F080402A
:100B00000C499839C1F898000846D0F8980040F090
:100B10008240C1F898000848406D40F00400064942
:100B2000486506480860002048660867012088601C
:100B300070470000985006400060024001008000AD
:100B40008248006840F080408149C1F8240108468D
:100B5000D0F8280140F08040C1F828010846D0F8BC
:100B60002C0140F08040C1F82C010846D0F830013B
:100B700040F08040C1F830010846D0F8340140F020
:100B80008040C1F834017348406940F00400714965
:100B900048618815704988606E48406920F00800F7
:100BA0006C49486140F213106B49C8606948406D58
:100BB00040F00100674948658815684908600846A3
:100BC000406840F4407048600846806840F44070D7
:100BD00088600846C06840F44070C860604800689B
:100BE00040F440705E4908600846406840F4407038
:100BF00048600846806B40F4407088630846C06BCC
:100C000040F44070C8635748006840F4407055494C
:100C100008600846406840F44070486052480068E8
:100C200040F4A060504908604A48D0F8140140F0F0
:100C300002004E49086088154B4948604848806862
:100C400040F48060464988600846C06840F480608F
:100C5000C8604048D0F8940040F400703D49C1F8A5
:100C600094003F48406A40F480703D4948623948EA
:100C7000D0F8D40040F010003649C1F8D40039480B
:100C8000006940F48070374908613248D0F8D400D8
:100C900020F020003549403908604FF4897031490F
:100CA00048612C48D0F8D40040F400402949C1F8EC
:100CB000D4002C48C06B40F480702A49C863254892
:100CC000D0F8D40020F04000284940390860284876
:100CD000244988611F48D0F8140120F008002349F6
:100CE000086023482049C8600846006940F4C06095
:100CF00008611848D0F8140120F020001B49086052
:100D00004FF48970184948610846806940F4806052
:100D100088611048406C40F001000E494864084664
:100D2000D0F8040140F00200C1F804010846D0F8F0
:100D3000880040F40070C1F888000846D0F8C4006C
:100D400040F40040C1F8C400704700002451064040
:100D50000050064000F00F400090044000A0044006
:100D600000B0044000C0044000D0044014F10F4023
:100D700010010B00F0B5134600240AE00246157876
:100D8000521C16780E70491C0D70491C801C671C83
:100D9000FCB29C42F2DBF0BD10B52348C06840F0C5
:100DA00001002149C8602148006900F0040030B109
:100DB0001E48806840F004001C49886033E01B48EE
:100DC000406840F00400194948601948007801283B
:100DD00009D1002016490870FFF7A8FB15480078D4
:100DE000401C1449087014480078012801D1FFF70D
:100DF000ADFD1148007808B9FFF78EFD0F48007867
:100E000088B90F48007801280DD100F017FD0D4872
:100E1000007818B901200B49087004E00020094946
:100E2000087000F011F810BD0070034000F00F4092
:100E30000E80FF1FE481FF1F0080FF1F4680FF1F01
:100E4000DD81FF1FE781FF1F002104488162044804
:100E5000806840F0040002498860704700700340D9
:100E600000F00F400121014881627047007003408B
:100E70004FF48031054801600846054908600A21A1
:100E80000348001F80F830137047000084E200E040
:100E900004E100E04FF0C060094908600848DC3810
:100EA000D0F8DC0040F080400860012005498860EF
:100EB000086105480862012102488162704700000C
:100EC000DC500640007003400A8B0200002000BF87
:100ED00007494969C1F340010029F9D00449496F24
:100EE000C8B20349496941F00201014A51617047A2
:100EF00000C0024000BF0749496901F00101002913
:100F0000F9D004494866496941F00101014A51613B
:100F10007047000000C00240002000BF0749496937
:100F2000C1F340010029F9D00449496FC8B203490F
:100F3000496941F00201014A5161704700D0024005
:100F400000BF0749496901F001010029F9D00449AE
:100F50004866496941F00101014A5161704700004A
:100F600000D002404FF08050044908604FF0E0216B
:100F7000C1F80001082102480170704780E200E0DA
:100F80001CE400E030B50021634AD26D634B1A6067
:100F9000614A5269624B1A6000BF5F4A5269C2F3EC
:100FA0004002002AF9D05C4A52695E4B1A605A4AE4
:100FB000526942F00202584B5A611A46506F5A4A1F
:100FC00010605A4A127822B1012A1CD0022A7DD11F
:100FD00030E047F6F87290420FD10022544B1A705D
:100FE0001A4614781278521C1D462A70514A22F86B
:100FF000140001224D4B1A7004E000224B4B1A7072
:101000004B4B1A7085E04FF6FC7290420CD1484A67
:1010100014781278521C464D2A70464A22F8140061
:101020000222424B1A7004E00022404B1A70404BDF
:101030001A706EE047F6F872904233D04FF6FC72A9
:1010400090422FD03A4A14781278521C384D2A70A8
:10105000384A22F814002A461278622A57DB002107
:101060000AE08A1C334B33F81220C2F30C02324BD5
:1010700023F811204A1C91B26029F2DB60222F4B29
:101080001A7001222E4B1A700022294B1A70274B1E
:101090001A702C4A126842F010022A4BCC3BC3F85B
:1010A000CC2034E047F6F872904212D10022204B57
:1010B0001A7003461E4A14781278521C1C4D2A706E
:1010C0001C4A22F814300122184B00E020E01A706C
:1010D0001DE04FF6FC72904219D10022144B1A7099
:1010E00047F6F873124A14781278521C104D2A7081
:1010F000104A22F8143003462A4614781278521CFB
:101100002A700C4A22F814300222084B1A7000E0B0
:1011100000BF00BF30BD000000E002401080FF1F94
:101120001480FF1F1880FF1F0880FF1F0D80FF1F06
:101130000C80FF1FEC81FF1FEC82FF1F0F80FF1F41
:101140000E80FF1FCCF00F400020224908604FF0B6
:1011500046402049B839C1F8B80000201E4908614E
:101160001E480866022088610020C8610862486243
:1011700088650920086100201649091F08604FF0A2
:10118000464008600020164908618861C86108620D
:1011900001204862134808661348086403208865E4
:1011A0000920086100200B49083908604FF04640CB
:1011B000086000200D4908618861C861086201204B
:1011C00048620848086608480864032088650920C2
:1011D00008617047B850064000E002400F00001B55
:1011E00000D00240070000030808090400C00240C4
:1011F00005480649486100BF04480069C0F3036020
:101200000628F9D170470000120001060040064090
:101210004FF080410548016000070549086007213B
:101220000348001F80F83E137047000084E200E08E
:1012300004E100E010B50C48006800F0400090B1F7
:101240000948006840F040000749A039C1F8A000F3
:101250000648006800F0400028B1FFF71BFEFFF7CA
:1012600007FEFFF7FFFD10BDA0C00440D0F00F4007
:101270004448006800F00800002819D04148006880
:1012800040F008003F49A039C1F8A00001203E49C4
:1012900008703E48007860B93D48006800F00800DA
:1012A00038B10120394908703A4840683A49086025
:1012B00066E03648007801280CD13548006800F017
:1012C000080038B902203149087032484068334973
:1012D000086055E02D480078022851D12C4800685C
:1012E00000F0080000284BD0002028490870294849
:1012F00040682B49086028480068284909688842E6
:1013000007D92548006825490968401A2549086019
:101310000EE02148006821490968884208D21F4828
:101320000068C0F1FF301C49096808441D49086085
:10133000194800681A490968884207D916480068A0
:1013400017490968401A184908600EE012480068F9
:1013500013490968884208D211480068C0F1FF307B
:101360000D4909680844104908600E4800684FF4A8
:101370007A7148430C490968B0FBF1F00B490880C9
:1013800070470000A0D004404A80FF1F4C80FF1F20
:1013900010F10F40006002405880FF1F5C80FF1F6B
:1013A0006080FF1F6480FF1F6880FF1F6C80FF1F2D
:1013B0002DE9F04104460E461546002746F0400050
:1013C0000F490870802040EA252048708D70002069
:1013D000C870087148718871012C05D1082209492B
:1013E000074800F059F806E0022C04D1082205490C
:1013F000034800F071F8034887793846BDE8F0816A
:10140000EC87FF1F2C88FF1F40F202200D49086067
:1014100034200D49C1F8080100BF0A48001F0068C8
:1014200000F400000028F8D101200649091F0860D7
:1014300000BF0448001F006800F080700028F8D04A
:1014400070470000044106400040064000BF1048BD
:10145000006800F400000028F9D10D49086040F24E
:101460000230091D08600B48091D086000BF0848CC
:10147000006800F400000028F9D101200449086048
:1014800000BF0348006800F080700028F9D0704762
:101490000046064000011800F0B505460E46174606
:1014A0000C48806C40F001000A498864002308E081
:1014B000E85CFFF71FFDFFF709FD0446F454581CD4
:1014C000C3B2BB42F4DB0348406C40F00100014969
:1014D0004864F0BD00F00F40F0B505460E461746D3
:1014E0000E48006840F002000D49C1F808010023D1
:1014F00008E0E85CFFF724FDFFF70EFD0446F45416
:10150000581CC3B2BB42F4DB0448001F006840F023
:1015100002000349C1F80401F0BD000008F10F40CA
:1015200000F00F4010B500F097FA73480069734857
:101530000088401C7149088071480078012806D154
:1015400000206F4908706F4908706C4908806B482B
:101550000088642809DB0020684908800120694967
:1015600008704FF47A70684908806348D03000688A
:1015700000F0200090B165480088401C6349088055
:10158000002063490880614800880A2818DB012090
:10159000604908700A205D49088011E05C480088B5
:1015A000401C5B4908800020584908805848008842
:1015B0000A2805DB0020574908700A205449088092
:1015C0005548006800F0200088B154480088401C4D
:1015D000524908800020524908805048008801285C
:1015E00017DB01204F4908704C49088011E04C4836
:1015F0000088401C4A490880002048490880484823
:101600000088012805DB0020464908700120444974
:10161000088045480068401C434908600846006847
:1016200042490988884225D341480078E0B94149B8
:101630000878C11700EB91718910A0EB810119B1F5
:1016400064203A49088003E04FF47A7037490880F3
:1016500038480078401C3749087008460078082848
:1016600005DB0020087002E00020324908700020ED
:101670002D4908602048006900F00800B8B12E48E4
:101680000088401C2C49088008460088B0F5FA6F95
:1016900006DB0020294908804FF4FA6026490880BB
:1016A00000202749088001202649087014E02548B9
:1016B0000078012810D100201F49088020480088A8
:1016C000401C1F490880084600880A2804DB0A20BD
:1016D000088000201B4908701B480088401C1A49DC
:1016E0000880084600880A2804DB002008800220C1
:1016F00000F09CF910BD000000F00F404880FF1F73
:101700004A80FF1F4B80FF1F6C80FF1F4480FF1F1C
:101710004280FF1F4080FF1F10F10F403E80FF1FDF
:101720003C80FF1F3A80FF1F2480FF1F0280FF1FA5
:101730004780FF1F7680FF1F7280FF1F7480FF1F8E
:101740007080FF1F6F80FF1F3680FF1FF0B50021E4
:101750000125214E3669C6F30346741C1E4E3669B8
:10176000C6F30366012E06D0022E06D0032E0ED03D
:10177000062E26D113E0194925E0194E366806F0E9
:10178000010008B1174E00E0174E31461BE0174E1E
:10179000366806F00300164E56F8201013E00F4985
:1017A000144E3668C6F30226721C124E3668C6F313
:1017B000044606F1100301FB03F65700B6FBF7F1F0
:1017C00001E0002500BF00BF012D03D1B1FBF4F6FD
:1017D000094F3E60F0BD0000004006400024F400C8
:1017E0000842064000127A0080841E00084306402A
:1017F000681E000008460640E881FF1F0B4800688D
:1018000040F47000094908600948006820F08040F1
:10181000074908600748084948600846406842F29E
:10182000201008604FF6FF708860704788ED00E078
:1018300034EF00E020C528D90020054008B510226B
:1018400029492A48FFF796FA2020274B40220121F8
:101850000090084600F05AF810222349234820300F
:10186000FFF788FA2020204B40220221009001201F
:1018700000F04CF810221C491C484030FFF77AFA5F
:101880002020194B402203210090012000F03EF857
:101890001022154915486030FFF76CFA2020124BD2
:1018A000402201210090022000F030F810220E4961
:1018B0000E488030FFF75EFA20200B4B40220221B9
:1018C0000090084600F022F8102207490748A0308F
:1018D000FFF750FA2020044B402203210090022001
:1018E00000F014F808BD00002C8AFF1F6C85FF1F54
:1018F0000448054948604FF6FF7088604FF4045073
:101900000860704720C528D9002005402DE9F04720
:1019100006460F4690469946089C402C1FDA002C3C
:101920001DDD07F03F001849087008464470C8F3F1
:101930000620887081F80380002508E099F80010DF
:10194000281D114A115409F10109681CC5B2A542AC
:10195000F4DB0021201D0C4A1154601D1154E01CC1
:10196000384400F0FF0A012E05D1524607490648C7
:10197000FFF792FD06E0022E04D1524603490248C9
:10198000FFF7AAFDBDE8F087EC87FF1F2C88FF1F3B
:101990002DE9F04105460C4616461F4644F040002E
:1019A0000E490870C6F3062048708E700846C7704E
:1019B000002008714871012D06D1E01CC2B208490F
:1019C0000648FFF769FD07E0022D05D1E01CC2B211
:1019D00003490248FFF780FDBDE8F081EC87FF1F57
:1019E0002C88FF1F10B5002804DB0A07130E054AD8
:1019F000135406E00A07140E034A00F00F031B1FDE
:101A0000D45410BD00E400E018ED00E002E008C886
:101A1000121F08C1002AFAD170477047002001E068
:101A200001C1121F002AFBD1704700000449096858
:101A300021F01F01024A116000F01F011160704780
:101A400000B003400349086000BF0249096800294B
:101A5000FBD170471C80FF1F0448006820B1034879
:101A60000068401E01490860704700001C80FF1F8D
:101A700010B5002400BF09E02948035D2948025D34
:101A800001210846FFF784FF601CC4B2572CF3D332
:101A9000002409E02248035D2248025D0221012062
:101AA000FFF776FF601CC4B2572CF3D3002409E083
:101AB0001B48035D1B48025D03210120FFF768FFFF
:101AC000601CC4B2572CF3D3002409E01448035D12
:101AD0001448025D01210220FFF75AFF601CC4B2C6
:101AE000572CF3D3002409E00D48035D0D48025D37
:101AF00002210846FFF74CFF601CC4B2572CF3D3F9
:101B0000002409E00648035D0648025D0321022027
:101B1000FFF73EFF601CC4B2572CF3D310BD00008A
:101B2000D280FF1F7B80FF1F08B5104A1268009209
:101B300000210F4A0F4B9A4213D0002006E00D4AB5
:101B400052F820200A4B43F82020401C0A4A084B38
:101B5000D21AB0EB920FF2D31A465DF821301A6018
:101B600003E0044A5DF821301A6008BD641E0000DD
:101B700000000000000000000080FF1F10B53220B0
:101B8000FFF760FF1223002201210846FFF700FF44
:101B900000BF002201210846FFF70AFC1228F8D1F5
:101BA00000BF00BF1223002202210120FFF7F0FE38
:101BB00000BF002202210120FFF7FAFB1228F8D112
:101BC00000BF00BF1223002203210120FFF7E0FE27
:101BD00000BF002203210120FFF7EAFB1228F8D101
:101BE00000BF00BFFEF788FFFEF77EFF00F008F998
:101BF000A323A12201210846FFF7CAFEA323A122A5
:101C000002210120FFF7C4FEA323A122032101200A
:101C1000FFF7BEFEA12201210846FFF7C9FBA3235F
:101C2000A12201210220FFF7B3FEA323A12202215A
:101C30000846FFF7ADFEA323A12203210220FFF7F0
:101C4000A7FEFFF715FF0023A12201210846FFF799
:101C50009FFE0023A12202210120FFF799FE00230D
:101C6000A12203210120FFF793FEA12201210846B2
:101C7000FFF79EFB0023A12201210220FFF788FE2F
:101C80000023A12202210846FFF782FE0023A122A1
:101C900003210220FFF77CFE00239A22012108463F
:101CA000FFF776FE00239A2202210120FFF770FE43
:101CB00000239A2203210120FFF76AFE9A220121C4
:101CC0000846FFF775FB00239A2201210220FFF747
:101CD0005FFE00239A2202210846FFF759FE0023E7
:101CE0009A2203210220FFF753FE6420FFF7AAFE89
:101CF0001323002201210846FFF74AFE1323002286
:101D000002210120FFF744FE1323002203210120BA
:101D1000FFF73EFE002201210846FFF749FB13238F
:101D2000002201210220FFF733FE132300220221AB
:101D30000846FFF72DFE1323002203210220FFF7A0
:101D400027FE3220FFF77EFE00BF4FF4A172012173
:101D50000846FFF72DFB0428F7D100BF00BF00BFE6
:101D60004FF4A17202210120FFF722FB0428F7D1D2
:101D700000BF00BF00BF4FF4A17203210120FFF795
:101D800017FB0428F7D100BF00BF012001490870EC
:101D900010BD0000DD81FF1F0124FFF7A9FDFFF743
:101DA00033FBFFF753FBFFF723FAFFF7CFFC00F0FD
:101DB00031F8FEF7C5FEFFF7C7F9FFF7D3F8FEF7D6
:101DC0008BFBFFF725FA9220FFF73CFE0A480068DC
:101DD00040F4007008498439C1F884000AE0012CFD
:101DE00006D106480078012802D1FFF7C7FE00247B
:101DF000FEF7CCFDF3E7000084F00F403A80FF1FB0
:101E00000348006840F0180001490860704700006E
:101E10000060024010B5124800684FF47A71B0FBC0
:101E2000F1F4601EB0F1807F01D301200FE0601E4D
:101E30004FF0E02148610F214FF0FF30FFF7D2FD56
:101E400000204FF0E021886107200861002008B1E0
:101E500000BFFEE70021481EFFF7C4FD10BD0000D3
:101E6000E881FF1F08ED00E0006CDC02007519033B
:101E7000007E560300879303981E00000080FF1F1A
:101E8000EC010000800400006C1F0000EC81FF1FCB
:101E9000BC0800001C1A0000210236C8BA01070164
:101EA000259BE8032F12011058090A0B0C0D0E0F89
:101EB000101112131415161718898A8B8C8D8E8F9A
:101EC000909192939495969798191A2122232425FC
:101ED000262728292A2B2C2D2E2F30313234353726
:101EE000404142434445464748494A4B4C4D4E4F7A
:101EF000505152535455565758595A5B5C5D5E5F6A
:101F0000D0100F1E2E3D4C5C6B7A8A99A8B8CADFA0
:101F1000E7200E1D101BFFFF1213306075B2F26632
:101F200012E717FF5B2A61FF230D1C10300D04021E
:101F30001110100F1F2F3F4F5F6F7F8F9FAFBFCFCD
:101F4000DFEFCA1F012957273F607FFFF0FF2264A0
:101F5000141B2A611A03570B1C03E802095557D6B4
:0C1F600043405DC05F0400D8B8050000DD
:0400000500000411E2
:00000001FF
